:100000000C94C9020C9410030C9410030C9410036C
:100010000C9410030C9410030C9410030C94100314
:100020000C9410030C9410030C943A0C0C940C0DCB
:100030000C9410030C9410030C9410030C941003F4
:100040000C9410030C94A0210C9410030C94100336
:100050000C9410030C94321B0C9410030C9410039A
:100060000C9410030C9410030C9410030C941003C4
:100070000C9410030C9410030C9410030C941003B4
:100080000C9410030C9410030C9410030C941003A4
:100090000C9410030C9410030C9410030C94100394
:1000A0000C9410030C9410030C941003790D9B0D09
:1000B0008E0E9B0D8E0EE00D030E8E0E580E6B0EE7
:1000C0005A115A1189118911CC11061213141314E3
:1000D0001F12131414131413E71313141314FE1321
:1000E00075FF01E20157025701620262016202627A
:1000F00001040204015B025B02E2000000F0A1F0D7
:10010000A2F0A329002B00E300E100E00000001EA4
:1001100000140004001D7406014E001F001A001692
:10012000001B0019012A00200008000700060050EB
:1001300000280021001500090019004F004B002283
:100140000017000A0005000000C30023002F000074
:10015000004A0000003E002400300000004D000076
:10016000003B0025001C000B0011000000C200260F
:100170000018000D0010005100490027000C000E6F
:1001800000360052002C002D0012000F0037000036
:100190007FC1002E0013003300380035004C002AC8
:1001A0000031003400E500E400000001000100011E
:1001B000000100010000003A001E0220022202039A
:1001C0003001003B001F0221022302010001003C1C
:1001D000002F0226022F00010001003D00300227FF
:1001E000023000010001003E0031023500350200FE
:1001F0000001003F0001000000010000000100407C
:100200000001000000010000000100410052005107
:10021000002402000001004200240021001E000111
:100220000001004300250022001F003700010044A8
:100230000026002300200027000100450025022E93
:100240000231002E004C0546000100010001003D76
:100250000400000050010001000100010000000145
:10026000000100010001000100010001000100F295
:10027000000100010001000100F000F1000100F4A4
:1002800000010001000100F3000100F50001000180
:100290000001000100010000000100010001000058
:1002A0000001000000010001000100000001000049
:1002B0000001000100010001000100000001000137
:1002C00000010001000100AA00010001000100017D
:1002D00000AC00A900B600010001000100AB00A8BD
:1002E0000001000100010001000100010001000106
:1002F000000100AE00010001000000E200E200E2A7
:1003000000E200E20000005900010004000100E2E8
:100310000001005A00010001000100E200E2005B60
:10032000000800070006000100E2005C000100096F
:10033000000100010001005D000100010005000056
:100340000001005E00010000000100000001005FEC
:100350000001000000010000000100600001000138
:100360000001000000010061005F005C00590062B4
:10037000000100620060005D005A006200E2005768
:100380000061005E005B006200E20057005700570A
:1003900000570057000100010001000100010001A9
:1003A00000000016034500720067006F0044006FF4
:1003B000007800200045005A000000160345007236
:1003C0000067006F0044006F007800200045005A6D
:1003D0000000000403090409026D00040100A0FAF2
:1003E000090400000103010100092111010001229B
:1003F0003F000705810308000A0904010001030109
:100400000200092111010001224D000705820308A5
:10041000000A090402000103000000092111010083
:10042000012236000705830308000A0904030001BE
:100430000300000009211101000122390007058491
:10044000031000011201100100000008EDFE071367
:1004500001000102000105010906A101050719E0DB
:1004600029E7150025019508750181020508190184
:1004700029059505750191029501750391010507FF
:100480001900297715002501957875018102C005AD
:10049000010980A101850216010026B7001A01009A
:1004A0002AB700751095018100C0050C0901A10152
:1004B0008503160100269C021A01002A9C02751071
:1004C00095018100C005010902A1010901A10005F2
:1004D0000919012905150025019505750181029568
:1004E00001750381010501093009311581257F95C9
:1004F000027508810609381581257F9501750881E7
:1005000006050C0A38021581257F950175088106BC
:10051000C0C005010906A101050719E029E715007A
:10052000250195087501810295017508810105086D
:100530001901290595057501910295017503910130
:100540000507190029FF150025FF9506750881008C
:10055000C0000000000000000000000001020406CE
:100560000A0F17202C3A4A5D71879DB3C7DAE9F567
:10057000FCFFFCF5E9DAC7B39D87715D4A3A2C2090
:10058000170F0A060402010000000000000000002E
:10059000000011241FBECFEFDAE0DEBFCDBF04B6EE
:1005A00003FE27C08091EE019091EF01A091F00130
:1005B000B091F1018730904BA740B04BD1F410922D
:1005C000EE011092EF011092F0011092F10114BEB1
:1005D00084B7877F84BF0FB6F894A8958091600098
:1005E000886180936000109260000FBEE0E0FFE33E
:1005F000099511E0A0E0B1E0E2EEF6E402C005905A
:100600000D92A433B107D9F721E0A4E3B1E001C012
:100610001D92AE3EB207E1F70E9481090C946F2350
:100620000C940000CF93DF93EC01662319F0633044
:1006300059F00DC08A81882321F085EE0E94EF0FCA
:1006400003C085EE0E94B7108A81811103C080E04B
:1006500090E002C080EE90E0DF91CF910895089580
:100660006091B1017091B2018091B3019091B40198
:100670000E945F1A56985E9825982D9826982E9875
:1006800027982F98823039F0833041F0813041F43F
:10069000259A2D9A0895269A2E9A0895279A2F9A88
:1006A00008950C94300356985E9825982D982698B6
:1006B0002E9827982F988FEF90E090938900809341
:1006C000880090938B0080938A0090938D00809394
:1006D0008C00259A2D9A2FEF80E792E021508040E0
:1006E0009040E1F700C00000269A2E9A2FEF80E795
:1006F00092E0215080409040E1F700C00000279A2E
:100700002F9A2FEF80E792E0215080409040E1F750
:1007100000C0000025982D982FEF80E792E021502F
:1007200080409040E1F700C0000026982E982FEFFF
:1007300080E792E0215080409040E1F700C0000047
:1007400027982F9856985E9825982D9826982E9839
:1007500027982F98089589EA8093800089E08093F4
:10076000810024982C983F988AB18F748AB96E982A
:10077000479A8BB1806B8BB9769A0E9453030C9485
:100780002F0380E2809300018091340181110EC01B
:100790000E94100481E0809334012FEF83ED90E3F9
:1007A000215080409040E1F700C0000080E40E94AA
:1007B00016048093000181112EC00E944004809392
:1007C0000001811128C00E94400480930001811122
:1007D00022C08FE30E9440048093000181111BC05E
:1007E0000E94380480E40E94160480930001811165
:1007F00012C08CE00E9440048093000181110BC064
:100800000E94400480930001811105C08FE30E9483
:100810004004809300010E943804809100010895F3
:100820001092B9008AE08093B800089594EA9093FA
:10083000BC009091BC0097FFFCCF9091B900987FCD
:10084000983021F0903111F081E008958093BB0041
:1008500084E88093BC008091BC0087FFFCCF80912E
:10086000B900887F883111F0803471F780E00895F5
:1008700084E98093BC008091BC0084FDFCCF089586
:100880008093BB0084E88093BC008091BC0087FF0C
:10089000FCCF9091B900987F81E0983209F480E014
:1008A000089584E88093BC008091BC0087FFFCCF52
:1008B0008091BB00089580910001811115C080E4F2
:1008C0000E9416048093000181110CC082E10E94F5
:1008D000400480930001811105C08FEF0E94400405
:1008E000809300010E94380484B1807F84B985B16F
:1008F000807F85B98AB1837F8AB98BB1837F8BB9B9
:100900003E98469808950E94C103809300010E947A
:100910005B0480B38C7080BB81B3836F81BBE4E4E4
:10092000F1E0A6E3B1E011921D9281E0E235F80713
:10093000D1F70C94AB039F92AF92BF92CF92DF920C
:10094000EF92FF920F931F93CF93DF93809100015B
:10095000882379F0809135018F5F80933501811173
:1009600008C00E94C10380930001811102C00E944F
:10097000530386E3E82E81E0F82E8701C0E0D0E043
:10098000BB24B39492E0A92ECC24C394D12CC730BD
:10099000D10500F580910001811164C080E40E94BE
:1009A000160480930001811112C082E10E9440046C
:1009B0008093000181110BC0C6010C2E01C0880F6D
:1009C0000A94EAF780950E944004809300010E94F7
:1009D000380448C0CA30A1F028F4C83059F0C930F2
:1009E00061F005C0CC3089F070F0CD3089F0209AEC
:1009F000289810C0219A29980DC0229A2A980AC0D6
:100A0000239A2B9807C0529A01C0539A5B9802C050
:100A10003E9A4698E0EAEA95F1F78FB181708B250E
:100A2000799902C032E001C030E0832B7C9902C08A
:100A300034E001C030E0832B7D9902C028E001C082
:100A400020E0822B7E9902C090E101C090E0892BCA
:100A50009FB19095991F9927991F9295990F907E14
:100A6000892B0FC08091000181114AC080E40E944F
:100A7000160480930001882381F1912C0E94380490
:100A8000892DD8019C91981719F08C93A09201019F
:100A90000E945B0421960F5F1F4FCE30D10509F0F5
:100AA00076CF80910101882369F181508093010103
:100AB000882339F0EFE9FFE03197F1F700C000003B
:100AC00021C0E4E4F1E0D7018D917D018193B4E48C
:100AD000EB16B1E0FB06B9F715C083E10E944004B4
:100AE000809300018111C9CF81E40E941604809394
:100AF00000018111C2CF0E945104982E9094BECF64
:100B000080E0BFCF0E94510381E0DF91CF911F9120
:100B10000F91FF90EF90DF90CF90BF90AF909F909C
:100B20000895E82FF0E0EC5BFE4F80810895089572
:100B30008B3B910580F4883A910548F5853A9105FB
:100B4000D8F48430910508F0B2C0019709F06EC066
:100B500081E090E00895803E910508F467C0883EEA
:100B6000910508F4A4C09C01205F310920313105B2
:100B700008F05CC090650895853A910509F459C064
:100B8000863A910509F058C082E890E40895883AC1
:100B9000910509F454C0893A910509F453C08A3A81
:100BA000910509F452C08B3A910509F451C08C3A71
:100BB000910509F450C08D3A910509F44FC0803B6E
:100BC000910509F44EC08E3A910509F44DC08F3A53
:100BD000910509F44CC0813B910509F44BC0823B5F
:100BE000910509F44AC0833B910509F449C0843B4F
:100BF000910509F448C0853B910509F447C0863B3F
:100C0000910509F446C0873B910509F445C0883B2E
:100C1000910509F444C0893B910509F443C08A3B1E
:100C2000910509F442C080E094E4089580E090E0EA
:100C3000089581E890E4089583E890E4089582EEB1
:100C400094E4089589EE94E408958AEE94E4089576
:100C500085EB94E4089586EB94E4089587EB94E49F
:100C600008958CEC94E408958DEC94E4089583E861
:100C700095E408958AE895E4089582E995E4089555
:100C800084E995E4089581E296E4089583E296E488
:100C9000089584E296E4089585E296E4089586E254
:100CA00096E4089587E296E408958AE296E408952A
:100CB000089524E5829FC0011124FC0126E0729F63
:100CC000E00DF11D1124E60FF11DEE0FFF1FED5F8A
:100CD000FE4F859194910895880F991FFC01E55866
:100CE000F040859194910895880F991FFC01E5507B
:100CF000FF4F85919491089524E5829FC0011124AE
:100D0000FC0146E0749FE00DF11D1124E60FF11D7A
:100D1000EE0FFF1FED5FFE4F859194919C013A9578
:100D200021154FE1340708F425C13F512115304109
:100D300020F49F700E94740608959C013053211581
:100D4000304118F49927906C0895811520E5920799
:100D500069F40E9437144FEF84E39CE041508040D7
:100D60009040E1F700C000000C94571B813020E553
:100D7000920731F48091CD0181608093CD01089577
:100D80009C0130552115304108F05CC0292F3327D4
:100D90002F70332721303105E9F4AC0164E0440FB2
:100DA000551F6A95E1F744275370BC01637077279C
:100DB00002C0220F331F6A95E2F73C68242B352BC3
:100DC00073E0880F991F7A95E1F780769927822B37
:100DD000932B08952230310529F4982F8827816FAD
:100DE000906A089523303105A1F4AC0133E0440F3B
:100DF000551F3A95E1F7407E57708370992721E09F
:100E000030E002C0220F331F8A95E2F7C9019C68C7
:100E100016C02430310531F5AC0123E0440F551FD5
:100E20002A95E1F7407E57708370992721E030E0E2
:100E300002C0220F331F8A95E2F7C9019A68842BFA
:100E4000952B08959C0130572115304118F49F705F
:100E5000906208959C0130582115304118F49F701C
:100E6000906A0895803E9105E0F4803C910558F524
:100E70008133910509F46FC048F48932910509F472
:100E800063C08A32910509F46DC072C0893391053F
:100E9000E9F082389105D1F08533910509F44DC010
:100EA00067C0833E910581F138F4803E9105B9F029
:100EB000823E9105D9F05CC0863E910561F1873E86
:100EC0009105A1F155C00E946C0608952091DF01A3
:100ED00020FD02C021FF4CC080EE90E049C080910F
:100EE000DF0180FFF9CF89E390E042C08091DF010C
:100EF00082FF0EC08091DF0184FF03C080E090E09C
:100F000037C083EE90E034C08091DF0182FFF2CFE2
:100F100082EE90E02DC08091DF0183FF0BC08091B5
:100F2000DF0184FDEBCF87EE90E022C08091DF01EE
:100F300083FFF5CF86EE90E01BC08091DF0185FF37
:100F400007C089E290E014C08091DF0185FFF9CFEE
:100F500085E390E00DC08091DF0186FF07C08AE243
:100F600090E006C08091DF0186FFF9CF81E390E039
:100F70000E949805089508950C94BB078091620122
:100F80000895CF93DF9300D01F92CDB7DEB79C01B9
:100F90008091E501843019F593E099833B832A839E
:100FA0009093E9008FEF9091E800815095FD06C085
:100FB00095ED9A95F1F700008111F5CF8091E80049
:100FC00085FF0DC040E050E063E070E0CE01019687
:100FD0000E942E0A8091E8008E778093E8000F909F
:100FE0000F900F90DF91CF910895CF93DF9300D0B2
:100FF0001F92CDB7DEB72091E501243021F522E024
:1010000029839B838A8383E08093E9008FEF90910B
:10101000E800815095FD06C095ED9A95F1F7000026
:101020008111F5CF8091E80085FF0DC040E050E0D0
:1010300063E070E0CE0101960E942E0A8091E800E4
:101040008E778093E8000F900F900F90DF91CF91F3
:1010500008959C018091E5018430F9F482E0809349
:10106000E9009FEF8091E800915085FD06C085ED75
:101070008A95F1F700009111F5CF8091E80085FF86
:101080000CC040E050E065E070E0C9010E942E0A0B
:101090008091E8008E778093E8000895CF93DF93E6
:1010A000EC018091E501843009F046C090910C017B
:1010B0009923D9F090910D019923B9F08093E9001B
:1010C0008FEF9091E800815095FD06C095E19A95CB
:1010D000F1F700008111F5CF8091E80085FF2CC069
:1010E00040E050E060E170E017C081E08093E900EB
:1010F0008FEF9091E800815095FD06C095ED9A958F
:10110000F1F700008111F5CF8091E80085FF14C050
:1011100040E050E068E070E0CE010E942E0A80912D
:10112000E8008E778093E80080E1FE01A2E5B1E05F
:1011300001900D928A95E1F7DF91CF91089580910A
:10114000E401811109C00E94BF0B0E941C0C809118
:10115000E20084608093E20008951092E401089513
:1011600008950C948D210E94ED1A0E9493210E94F3
:10117000C70E0C94BC0742E061EC81E00E94380B82
:1011800042E061EC82E00E94380B42E061EC83E0D7
:101190000E94380B42E161EC84E00C94380B8091A2
:1011A000E701833009F455C030F4813071F08230AA
:1011B00009F48EC008958A3009F47AC08B3009F49E
:1011C00060C0893009F09CC020C08091E601813A5E
:1011D00009F096C08091E800877F8093E8008091B5
:1011E000EA019091EB01892B21F460E182E591E025
:1011F00003C060E080E090E070E00E94790A809196
:10120000E8008B778093E80008958091E6018132B1
:1012100009F076C08091EA019091EB01009719F0F6
:10122000039709F06DC08091E800877F8093E80004
:101230008091E80082FD05C08091E5018111F8CF21
:101240005FC08091F100809362018091E8008B770C
:1012500053C08091E601813A09F052C08091EA01C1
:101260009091EB01892B09F04BC08091E800877FBA
:101270008093E8008091E80080FFFCCF80910C0112
:1012800036C08091E6018132D9F58091EA019091D2
:10129000EB01892BA9F58091E800877F8093E80016
:1012A0000E946D0B8091E80180930C010C9437141F
:1012B0008091E601813221F58091E800877F80935B
:1012C000E8000E946D0B8091E9018093630108950D
:1012D0008091E601813AA1F48091E800877F8093B4
:1012E000E8008091E80080FFFCCF8091630180934B
:1012F000F1008091E8008E778093E8000C946D0BEC
:10130000089584B7877F84BF0FB6F894A89580911D
:101310006000886180936000109260000FBE90E0D2
:1013200080E80FB6F89480936100909361000FBE3F
:101330000E94160F0E94BF0B0E941C0C8091E200BD
:1013400084608093E20078940E94A70E0E94180F98
:1013500082E091E00E94C20E0E947B218091E50113
:10136000853069F40E94AF1A8091E3018823B1F3BC
:101370000E94D91A882391F30E94180AEFCF0E9485
:101380001E0FECCF292F332723303105C9F060F42D
:101390002130310581F02230310509F041C08DE660
:1013A00090E027ED33E040C021323105E1F02232F8
:1013B000310531F135C082E190E024E434E034C0FD
:1013C00099278130910549F028F0029749F5E3EA21
:1013D000F3E005C0E3EDF3E002C0EBEBF3E0849152
:1013E00090E09F0121C06430D8F4E62FF0E0EE0FCA
:1013F000FF1FEE5DFE4F2081318189E090E014C037
:10140000643070F470E0FB01EE0FFF1FE65EFE4FEC
:1014100020813181FB01EA5EFE4F808190E004C0B3
:1014200080E090E020E030E0FA01318320830895ED
:1014300080E189BD82E189BD09B400FEFDCF8091C4
:10144000D8008F7D8093D8008091E00082608093E7
:10145000E0008091E00081FDFCCF0895CF92DF9203
:10146000EF92FF920F931F93CF93DF93EC018B01C9
:101470006A010E948C0B811133C0C114D10439F070
:10148000F60180819181081B190BC80FD91FE12C2F
:10149000F12C0115110519F18091E80085FD16C0A8
:1014A0008091E8008E778093E800C114D10449F060
:1014B000F60180819181E80EF91EF182E08285E0DB
:1014C0000FC00E948C0B882321F30AC0899180935E
:1014D000F10001501109FFEFEF1AFF0ADACF80E0A7
:1014E000DF91CF911F910F91FF90EF90DF90CF9000
:1014F00008952091EC013091ED012617370748F04F
:101500006115710539F42091E8002E772093E800E9
:1015100001C0B901FC0120E06115710579F18091EC
:10152000E5018823F1F18530F1F18091E80083FD38
:101530003CC08091E80082FD2EC08091E80080FFD1
:10154000EBCF2091F3008091F20090E0922B611597
:10155000710551F08830910538F421912093F10004
:10156000615071090196F3CF21E0089709F020E05E
:101570008091E8008E778093E800CECF2111CFCF05
:101580000AC08091E501882361F0853061F0809187
:10159000E80083FD0AC08091E80082FFF2CF80E07E
:1015A000089582E0089583E0089581E008952091F0
:1015B000EC013091ED012617370748F061157105F0
:1015C00039F42091E8002E772093E80001C0B9019A
:1015D000FC0120E06115710591F18091E5018823FE
:1015E00009F440C0853009F43FC08091E80083FDD4
:1015F0003DC08091E80082FD2FC08091E80080FF0F
:10160000E9CF2091F3008091F20090E0922B6115D8
:10161000710559F08830910540F424912093F10030
:101620003196615071090196F2CF21E0089709F0D7
:1016300020E08091E8008E778093E800CBCF2111E5
:10164000CCCF0AC08091E501882361F0853061F03C
:101650008091E80083FD0AC08091E80082FFF2CF0C
:1016600080E0089582E0089583E0089581E0089580
:10167000982F973068F59093E900981739F070919A
:10168000EC002091ED005091F00003C0242F762F44
:1016900050E021FD02C09F5FECCF3091EB003E7F18
:1016A0003093EB003091ED003D7F3093ED003091B1
:1016B000EB0031603093EB007093EC002093ED0071
:1016C0005093F0002091EE0027FDE5CF80E00895D3
:1016D0008F708093E90081E008958091E60187FF93
:1016E00011C08091E80082FD05C08091E501811163
:1016F000F8CF11C08091E8008B770BC08091E50195
:10170000882349F08091E80080FFF8CF8091E800BD
:101710008E778093E80008952091E4003091E500F1
:1017200095E64091EC00842F817040FF23C08091AA
:10173000E80080FD1DC08091E501882399F0853087
:1017400099F08091EB0085FD11C04091E40050912B
:10175000E5002417350729F3915011F09A01E1CFE4
:1017600084E0089582E0089583E0089581E008957B
:1017700080E008954091E80042FFDDCF08950E9487
:101780002D0C0E94350CE0EEF0E0808181608083BA
:10179000E8EDF0E080818F77808319BCA7EDB0E0A1
:1017A0008C918E7F8C9380818F7E80831092E40158
:1017B00008950F931F93CF93DF930E942D0C0E94E7
:1017C000350CC8EDD0E088818F7788838881806868
:1017D000888388818F7D888319BC1092E5011092DF
:1017E000E1011092E3011092E20100EE10E0F80135
:1017F00080818B7F808388818160888342E060E084
:1018000080E00E94380BE1EEF0E080818E7F8083E3
:10181000E2EEF0E080818160808380818860808357
:10182000F80180818E7F8083888180618883DF9149
:10183000CF911F910F910895E8EDF0E080818F7EA8
:101840008083E7EDF0E080818160808384E082BF67
:1018500081E08093E4010C94D90BE8EDF0E0808105
:101860008E7F80831092E20008951092DA00109229
:10187000E10008951F920F920FB60F9211242F933B
:101880003F934F935F936F937F938F939F93AF9308
:10189000BF93EF93FF938091E10082FF0BC0809193
:1018A000E20082FF07C08091E1008B7F8093E1001E
:1018B0000E94A60E8091DA0080FF1FC08091D800A0
:1018C00080FF1BC08091DA008E7F8093DA008091C8
:1018D000D90080FF0DC080E189BD82E189BD09B4D6
:1018E00000FEFDCF81E08093E5010E949F0805C0C6
:1018F00019BC1092E5010E94AD088091E10080FFC3
:1019000019C08091E20080FF15C08091E2008E7FB7
:101910008093E2008091E20080618093E2008091F8
:10192000D80080628093D80019BC85E08093E501DF
:101930000E94B1088091E10084FF30C08091E200F4
:1019400084FF2CC080E189BD82E189BD09B400FE1D
:10195000FDCF8091D8008F7D8093D8008091E100E9
:101960008F7E8093E1008091E2008F7E8093E20081
:101970008091E20081608093E2008091E101882300
:1019800011F084E007C08091E30087FD02C081E090
:1019900001C083E08093E5010E94B3088091E100DB
:1019A00083FF29C08091E20083FF25C08091E10080
:1019B000877F8093E10082E08093E5011092E1014E
:1019C0008091E1008E7F8093E1008091E2008E7F24
:1019D0008093E2008091E20080618093E20042E027
:1019E00060E080E00E94380B8091F0008860809376
:1019F000F0000E94B008FF91EF91BF91AF919F91CD
:101A00008F917F916F915F914F913F912F910F90A7
:101A10000FBE0F901F9018951F920F920FB60F9246
:101A200011242F933F934F935F936F937F938F93E3
:101A30009F93AF93BF93CF93DF93EF93FF93C091A7
:101A4000E900CF708091EC00D82FD17080FDD0E8F4
:101A50001092E9008091F000877F8093F0007894E5
:101A60000E94500D1092E9008091F00088608093F0
:101A7000F000CD2BCF70C093E900FF91EF91DF9183
:101A8000CF91BF91AF919F918F917F916F915F9116
:101A90004F913F912F910F900FBE0F901F9018956F
:101AA0001F93CF93DF93CDB7DEB7AA970FB6F89405
:101AB000DEBF0FBECDBFE6EEF1E08091F100819375
:101AC00021E0EE3EF207C9F70E94CF088091E800BE
:101AD00083FF24C18091E6019091E701492F50E0F6
:101AE0004A30510508F01AC1FA01EA5AFF4F0C9426
:101AF0002423803881F0823809F010C18091EA01F6
:101B00008F708093E9008091EB0085FB882780F936
:101B10001092E90006C08091E2019091E3019111D9
:101B200082609091E800977F9093E8008093F100A5
:101B30001092F100C8C0282F2D7F09F0EFC0882334
:101B400019F0823061F0EAC08091E801813009F03B
:101B5000E5C0933009F080E08093E3012BC08091D1
:101B6000E801811127C08091EA018F7009F4D6C085
:101B70008093E9002091EB0020FF1CC0933021F4FA
:101B80008091EB00806214C09091EB009061909383
:101B9000EB0021E030E0A90102C0440F551F8A95F7
:101BA000E2F74093EA001092EA008091EB0088602F
:101BB0008093EB001092E9008091E800877F86C057
:101BC0008111ACC01091E8011F778091E30080780B
:101BD000812B8093E3008091E800877F8093E80069
:101BE0000E946D0B8091E80080FFFCCF8091E300A4
:101BF00080688093E300111102C082E001C083E09D
:101C00008093E5018BC08058823008F087C08091B6
:101C1000E8019091E9018C3D53E0950779F583E067
:101C20008A838AE289834FB7F894DE01139620E015
:101C30003EE051E2E32FF0E050935700E49120FFA3
:101C400003C0E295EF703F5FEF708E2F90E0EA30B7
:101C500010F0C79601C0C0968D939D932F5F2431DD
:101C600049F74FBF8091E800877F8093E8006AE2E0
:101C700070E0CE0101960E94790A14C0AE014F5F58
:101C80005F4F6091EA010E94C209BC01892B09F4EF
:101C900045C09091E800977F9093E80089819A81F0
:101CA0000E94D70A8091E8008B778093E80036C0C5
:101CB0008038A1F58091E800877F8093E8008091CB
:101CC000E1018093F1008091E8008E778093E80035
:101CD0000E946D0B23C0811121C08091E801909179
:101CE000E90199270297D4F48091E800877F8093D7
:101CF000E8008091E8018093E1010E946D0B8091E2
:101D0000E101811106C08091E30087FD02C081E0FE
:101D100001C084E08093E5010E94BB088091E80047
:101D200083FF0AC08091E800877F8093E80080915C
:101D3000EB0080628093EB00AA960FB6F894DEBFAA
:101D40000FBECDBFDF91CF911F9108950895CF931E
:101D50008091E5018823A1F0C091E900CF709091B6
:101D6000EC00892F817090FD80E8C82B1092E9006B
:101D70008091E80083FD0E94500DCF70C093E90070
:101D8000CF91089590936901809368010895E0913F
:101D90006801F0916901309721F00190F081E02D08
:101DA000099480E00895E0916801F091690130970D
:101DB00021F00280F381E02D09940895E0916801FB
:101DC000F0916901309721F00480F581E02D0994AC
:101DD000089520916601309167012817390771F045
:101DE0009093670180936601E0916801F091690129
:101DF000309721F00680F781E02D09940895209115
:101E00006401309165012817390771F090936501DD
:101E100080936401E0916801F0916901309721F0AD
:101E20000084F185E02D0994089508950C94150F10
:101E30000E94F31A0E9483040C94B91BCF92DF9284
:101E4000EF92FF920F931F93CF93DF93CDB7DEB73F
:101E50002B970FB6F894DEBF0FBECDBF0E949B0438
:101E60008BE6C82E81E0D82E00E010E0E02E802F17
:101E70000E949105F60141916F01F82EF426B1F40C
:101E80000F5F1F4F0E30110589F78FEF89838A830B
:101E90001B820E94FC1A8160782F9D838C8349816C
:101EA0005A816B818D810E94C10F40C09091CD01FC
:101EB00091FF04C08B870E9497058B8520E030E05E
:101EC0004F2D50E0922FBA01022E02C075956795F2
:101ED0000A94E2F760FF24C02E83EF8221E030E015
:101EE000690102C0CC0CDD1C9A95E2F790E08C21D0
:101EF0009D21892B09F420E028870E94FC1A81602B
:101F0000782F9A8789874E815F8168858A850E94AC
:101F1000C10FF801E559FE4F8081C826C08206C076
:101F20002F5F3F4F2630310569F6AACF0E94A01ED1
:101F30000E94C70E90916A018917A1F00E94C70EF6
:101F400080936A012B960FB6F894DEBF0FBECDBF0B
:101F5000DF91CF911F910F91FF90EF90DF90CF9085
:101F60000C94BC072B960FB6F894DEBF0FBECDBF06
:101F7000DF91CF911F910F91FF90EF90DF90CF9065
:101F80000895CF93DF93CDB7DEB72B970FB6F894B4
:101F9000DEBF0FBECDBF4F83588769877A878B8797
:101FA000DE01119686E0FD0111928A95E9F785E040
:101FB000FE01379601900D928A95E1F749815A8189
:101FC0006B817C818D819E810E94CB162B960FB6F2
:101FD000F894DEBF0FBECDBFDF91CF910895CF93B0
:101FE000C82F882309F4C1C0823859F40E94C70E53
:101FF00081FDBBC089E30E9468190E94301A89E301
:102000000CC0833879F40E94C70E80FDAEC083E512
:102010000E9468190E94301A83E50E94A719CF9187
:102020000C94301A843859F40E94C70E82FD9DC06A
:1020300087E40E9468190E94301A87E4EECF8CEF83
:102040008C0F813A48F48C2F0E94E02081118DC0C2
:102050008C2F0E946819E3CF80E28C0F883048F4FF
:10206000C77081E001C0880FCA95EAF70E94E9199C
:10207000D6CF8BE58C0F833078F4C53A29F0C63A79
:1020800031F083E890E005C081E890E002C082E88A
:1020900090E0CF910C94E90E88E58C0F833108F025
:1020A00064C0C83A39F1C93A41F1CA3A49F1CB3A68
:1020B00051F1CC3A59F1CD3A61F1C03B69F1CE3AD8
:1020C00071F1CF3A79F1C13B81F1C23B89F1C33B58
:1020D00091F1C43B99F1C53BA1F1C63BA9F1C73BC6
:1020E000B1F1C83BB9F1C93BC1F1CA3BC9F180E0CC
:1020F00090E038C082EE90E035C089EE90E032C0CA
:102100008AEE90E02FC085EB90E02CC086EB90E04B
:1021100029C087EB90E026C08CEC90E023C08DECCA
:1021200090E020C083E891E01DC08AE891E01AC0E9
:1021300082E991E017C084E991E014C081E292E065
:1021400011C083E292E00EC084E292E00BC085E20F
:1021500092E008C086E292E005C087E292E002C009
:102160008AE292E0CF910C94FF0ECF9108958823DC
:1021700009F44BC0823859F40E94C70E81FF45C054
:1021800089E30E9468190E94301A89E30CC08338E1
:1021900071F40E94C70E80FF38C083E50E94681961
:1021A0000E94301A83E50E94A7190C94301A8438D3
:1021B00059F40E94C70E82FF28C087E40E94681964
:1021C0000E94301A87E4EFCF9CEF980F913A58F3B2
:1021D00090E2980F983050F4877091E001C0990F09
:1021E0008A95EAF7892F0E94EF19DFCF9BE5980FB8
:1021F000933020F480E090E00C94E90E885A83310B
:1022000020F480E090E00C94FF0E0895882321F0E4
:102210000E94E9190C94301A0895882321F00E9435
:10222000EF190C94301A0895BF92CF92DF92EF927B
:10223000FF920F931F93CF93DF9300D000D000D075
:10224000CDB7DEB77C0185E0F701DE011196019084
:102250000D928A95E1F7F70183819481892B09F426
:10226000E2C2908181818F3F19F49F3F09F4DBC264
:10227000F7010281258122952F7099838A838981B4
:102280009A812E830E942719182FB92E0E94261991
:102290000E94ED172E81002319F00E94061A2E814C
:1022A000EB2DE295EF704E2F50E0FA01E05AFF4F10
:1022B0000C9424238B2D807F9B2D9F70F92E8823D7
:1022C00019F0F29480EFF822002349F0FF2009F47E
:1022D00057C28F2D0E94F9190E94301A51C2812FC6
:1022E0000E94B710FF2009F49EC28F2D0E94FF1993
:1022F00026960FB6F894DEBF0FBECDBFDF91CF910B
:102300001F910F91FF90EF90DF90CF90BF900C94B2
:10231000301A3B2D307F8B2D8F70303211F082952B
:10232000807F112319F0113021F12CC00023B9F066
:10233000222309F490C1213009F08DC126960FB6F1
:10234000F894DEBF0FBECDBFDF91CF911F910F91EB
:10235000FF90EF90DF90CF90BF900C94191A22233A
:1023600019F0213009F45FC28E830E941C1A8E81FD
:1023700086C1002321F0223008F055C26CC1211122
:1023800052C27DC1002321F0222309F464C1F8C1A7
:10239000222309F474C109C28B2D8695869583701A
:1023A00019F08130D1F03FC2002321F0812F9B2D05
:1023B000937002C080E090E026960FB6F894DEBFDE
:1023C0000FBECDBFDF91CF911F910F91FF90EF9086
:1023D000DF90CF90BF900C94E90E002321F0812F65
:1023E0009B2D937002C080E090E026960FB6F89483
:1023F000DEBF0FBECDBFDF91CF911F910F91FF9038
:10240000EF90DF90CF90BF900C94FF0E812F0023B0
:1024100019F00E94A81D02C00E94101E26960FB639
:10242000F894DEBF0FBECDBFDF91CF911F910F910A
:10243000FF90EF90DF90CF90BF900C94951E8B2D66
:10244000837009F075C00111EEC1812F82958695C8
:102450008770880F880F912F9F70C92ED12CE12C87
:10246000F12C082E04C0CC0CDD1CEE1CFF1C0A94C1
:10247000D2F714FF12C00FE010E020E030E004C0FB
:10248000000F111F221F331F8A95D2F7C901B8010F
:10249000609570958095909503C060E070E0CB01E9
:1024A0004B2D4695469543704230C1F060F56C293E
:1024B0007D298E299F29413051F126960FB6F89437
:1024C000DEBF0FBECDBFDF91CF911F910F91FF9067
:1024D000EF90DF90CF90BF900C9414186C297D2959
:1024E0008E299F2926960FB6F894DEBF0FBECDBF6A
:1024F000DF91CF911F910F91FF90EF90DF90CF90E0
:10250000BF900C9430180E941418C701B60126968B
:102510000FB6F894DEBF0FBECDBFDF91CF911F91F4
:102520000F91FF90EF90DF90CF90BF900C94F81731
:10253000002319F08B2D817001C08695882309F442
:1025400072C1812F829586958770880F880F912F91
:102550009F70C92ED12CE12CF12C082E04C0CC0C7C
:10256000DD1CEE1CFF1C0A94D2F714FF12C00FE012
:1025700010E020E030E004C0000F111F221F331FC5
:102580008A95D2F7C901B8016095709580959095AC
:1025900003C060E070E0CB014B2D4695469543703B
:1025A0004230C1F060F56C297D298E299F29413088
:1025B00051F126960FB6F894DEBF0FBECDBFDF9166
:1025C000CF911F910F91FF90EF90DF90CF90BF9030
:1025D0000C94EE186C297D298E299F2926960FB61A
:1025E000F894DEBF0FBECDBFDF91CF911F910F9149
:1025F000FF90EF90DF90CF90BF900C940A190E944B
:10260000EE18C701B60126960FB6F894DEBF0FBECE
:10261000CDBFDF91CF911F910F91FF90EF90DF9091
:10262000CF90BF900C94D218103FD1F118F4103E07
:1026300050F4A1C0123F09F463C008F44CC0133F2A
:1026400009F473C098C01F708B2D8F710023A1F007
:102650000E946B18812F26960FB6F894DEBF0FBE2E
:10266000CDBFDF91CF911F910F91FF90EF90DF9041
:10267000CF90BF900C9406110E948C18812F269643
:102680000FB6F894DEBF0FBECDBFDF91CF911F9183
:102690000F91FF90EF90DF90CF90BF900C940D11B1
:1026A0000023A9F02111BFC08B2D8F7126960FB684
:1026B000F894DEBF0FBECDBFDF91CF911F910F9178
:1026C000FF90EF90DF90CF90BF900C94B118223024
:1026D00008F0A9C0E9CF0023A9F08B2D8F712696B1
:1026E0000FB6F894DEBF0FBECDBFDF91CF911F9123
:1026F0000F91FF90EF90DF90CF90BF900C946B18EC
:10270000002359F38B2D8F7126960FB6F894DEBFF8
:102710000FBECDBFDF91CF911F910F91FF90EF9032
:10272000DF90CF90BF900C948C18002399F08B2DE4
:102730008F7126960FB6F894DEBF0FBECDBFDF9126
:10274000CF911F910F91FF90EF90DF90CF90BF90AE
:102750000C94561826960FB6F894DEBF0FBECDBF68
:10276000DF91CF911F910F91FF90EF90DF90CF906D
:10277000BF900C944C180023A9F0222309F4ADCF8C
:10278000812F26960FB6F894DEBF0FBECDBFDF9126
:10279000CF911F910F91FF90EF90DF90CF90BF905E
:1027A0000C94EF0F222309F4ADCF812F26960FB69C
:1027B000F894DEBF0FBECDBFDF91CF911F910F9177
:1027C000FF90EF90DF90CF90BF900C94B7104B2DFF
:1027D0004F70612FC7010E94120326960FB6F8941E
:1027E000DEBF0FBECDBFDF91CF911F910F91FF9044
:1027F000EF90DF90CF90BF900C9470174B2D4F70DF
:10280000612FC70126960FB6F894DEBF0FBECDBF6D
:10281000DF91CF911F910F91FF90EF90DF90CF90BC
:10282000BF900C94580626960FB6F894DEBF0FBEE4
:10283000CDBFDF91CF911F910F91FF90EF90DF906F
:10284000CF90BF9008950E94061A0E94161A0E9407
:10285000DB190E94301A0E94451F0E94951E80E0DD
:1028600090E00E94E90E80E090E00C94FF0E0E9440
:10287000F6190C9423140E942719292F22952F70E2
:102880002C3030F42A3048F42250223078F405C03D
:102890002C3041F02F3031F009C0803E48F0803FAD
:1028A00029F406C093FB882780F9089580E00895F5
:1028B00081E00895CF93DF9300D000D01F92CDB771
:1028C000DEB70F900F900F900F900F90DF91CF9188
:1028D0000895CF93DF9300D000D000D0CDB7DEB7FE
:1028E00026960FB6F894DEBF0FBECDBFDF91CF9115
:1028F00008951F93CF93DF93C091790116E08091E3
:102900007A01C81799F0D0E01C9FF0011D9FF00DCF
:102910001124E558FE4F4081518162817381848189
:1029200095810E9469142196C770E9CFDF91CF91FC
:102930001F9108954091AB015091AC016091AD01A0
:102940007091AE018091AF019091B0010C94691427
:102950008091B00182958F7009F054C08091AD01D3
:10296000882309F44FC080917901A0917A014091A8
:10297000AE015091AF016091AB017091AC01B6E036
:102980008A1709F43FC090E041155105C1F17F3F1E
:1029900011F46F3FA1F1B89FF001B99FF00D112420
:1029A000E558FE4F218127132AC02081261327C016
:1029B0002281211124C0238134812417350710F48A
:1029C00021503109241B350B283C3105C0F42091DE
:1029D000B0012F7020612093B00126E0289FF00104
:1029E000299FF00D1124E058FE4F80818F70806187
:1029F00080838BEA91E00E9414110C947914019663
:102A00008770BECF0895CF92DF92EF92FF920F931F
:102A10001F93CF93DF93CDB7DEB762970FB6F894CD
:102A2000DEBF0FBECDBF8C0185E0F801DE011D9633
:102A300001900D928A95E1F7D8014C9111965C9125
:102A4000119712966C918091AE019091AF01009711
:102A500009F475C13091AB017091AC017F3F19F45D
:102A60003F3F09F46CC1F801C380D480E090AD0110
:102A7000EE2009F4BEC02091B001C816D90628F096
:102A8000D601A81BB90BCD0104C0809590958C0D83
:102A90009D1DFF24F394883C910578F0F12C207F54
:102AA00009F0C4C07C2DD98AC88A89890E945A1429
:102AB0008BEA91E00E941411AFC0822F807F09F051
:102AC00045C0571313C0431311C061110FC02F70BD
:102AD00020612093B0010E949A148BEA91E00E9439
:102AE00014118091B001F80185832EC0CD2819F111
:102AF0005F3F11F44F3FF9F0F62E61111CC0809139
:102B0000790120917A0136E0821709F45BC090E0E8
:102B1000389FF001399FF00D1124E558FE4F718167
:102B2000571306C07081471303C07281711103C02F
:102B300001968770E9CFF62E662309F41CC18091B7
:102B4000B00181608093B001F12C15C1571309C009
:102B5000431307C0611105C08091B001F80185835E
:102B6000C8C04D875E878D859E856A8B0E943B1409
:102B70006A898823D1F16623C1F12091B001822FA7
:102B800082958F7090E0029774F08091AB019091E4
:102B9000AC0198878F831986DB86CA862C87CE0185
:102BA00007960E94141186E0F801ABEAB1E00190AB
:102BB0000D928A95E1F70E94A8140E949A14FF24AE
:102BC000F394D9C04D875E878D859E850E94271915
:102BD000292F22952F70223008F0C1C09F7009F074
:102BE000BBC0805E883008F4C6C0C8010E941411C2
:102BF000E6CFC816D90608F453C0F601E81BF90B56
:102C0000CF01883C910508F450C0F12C7C2DD98A65
:102C1000C88A89890E945A14EBEAF1E086E0DF0154
:102C20001D928A95E9F70E949A14A5C0571314C003
:102C3000431312C0611110C08091B001F801858367
:102C4000C8010E94141186E0EBEAF1E0DF011D9259
:102C50008A95E9F7FE2C8FC04D875E878D859E850E
:102C60006A8B0E943B146A89882309F4BECF6623CD
:102C700009F4BBCF2091B001822F82958F7090E034
:102C800002970CF490CF8091AB019091AC019A83A4
:102C900089831B82DD82CC822E83CE01019681CF77
:102CA000809590958C0D9D1DACCFF62E662309F472
:102CB0009CCF571333C0431331C02091B00120FD86
:102CC00024C0822F82958F70482F50E04115510506
:102CD000E1F0D80115962C9315974F30510549F026
:102CE0008F5F982F9295907F822F8F70892B1596EA
:102CF0008C93C8010E94141186E0F801ABEAB1E0A0
:102D000001900D928A95E1F78ECF86E0F801ABEA4B
:102D1000B1E001900D928A95E1F72DC04D875E8755
:102D20008D859E850E943B1481113DCF8091B0011D
:102D300081608093B001C8010E9414111CC06623F9
:102D400009F453CF4D875E878D859E850E943B1485
:102D5000882309F44ACF27CF811143CF0CC02430F8
:102D600008F043CF9F7009F43CCFD80115969C9191
:102D7000907F09F036CF8F2D62960FB6F894DEBFA4
:102D80000FBECDBFDF91CF911F910F91FF90EF90BC
:102D9000DF90CF9008951F93CF93DF93CDB7DEB729
:102DA0002C970FB6F894DEBF0FBECDBF4F83588768
:102DB00069877A878B879C87CE0107960E940315C7
:102DC000882371F08A859B85892B09F441C0888509
:102DD0008F3F09F065C08F818F3F09F061C038C017
:102DE00086E0FE013796DE01119601900D928A95DC
:102DF000E1F76A857B856115710551F1FF81E885F1
:102E0000EF3F11F4FF3F21F120917A0130E0C90139
:102E10000196877099274091790150E084179507B2
:102E200009F447C0F983EA837D836C8396E0929F1F
:102E3000D001939FB00D1124A558BE4FFE013196CD
:102E400001900D929A95E1F780937A010E9479148E
:102E500016E08091790190917A018917B9F1189F54
:102E6000C001112485589E4F0E940315882371F1DB
:102E7000E09179011E9FF0011124E558FE4F408139
:102E8000518162817381848195810E94691480914E
:102E9000790190E001968770992780937901D9CFC5
:102EA0004F81588569857A858B859C850E94691438
:102EB000CFCF0E94371410927A0110927901EBEA79
:102EC000F1E086E0DF011D928A95E9F72C960FB6B6
:102ED000F894DEBF0FBECDBFDF91CF911F91089553
:102EE000EF92FF920F931F93CF93DF938C01892B67
:102EF00009F46CC0F12CEE24E394E8012196F8016A
:102F00008491843740F4843008F051C0813081F0DE
:102F1000823019F15BC0853709F444C0A8F19CE701
:102F2000980F903708F052C08F770E94B71041C0B9
:102F30000E5F1F4FFE01849190E2980F983050F47D
:102F40008770FE2D01C0FF0F8A95EAF78F2F0E9430
:102F5000091A14C00E94EF0F2DC00E5F1F4FFE0113
:102F6000849190E2980F983060F48770FE2D01C034
:102F7000FF0F8A95EAF78F2F0E940F1A0E94301ACE
:102F800019C00E94B71016C00E5F1F4FFE01C491FA
:102F9000CC2381F08FE99FE00197F1F700C000009A
:102FA000C150F6CF0E5F1F4FFE01F49003C00E9488
:102FB000EF0F8E018F2D882309F49FCFEFE9FFE0FB
:102FC0003197F1F700C000008150F5CFDF91CF912C
:102FD0001F910F91FF90EF90089508956093B501B0
:102FE0007093B6018093B7019093B8010C942314A9
:102FF0000F931F930091B5011091B6012091B70175
:103000003091B801DC01CB01802B912BA22BB32B8B
:103010008093B5019093B601A093B701B093B80126
:103020001F910F910C9423140F931F930091B501DE
:103030001091B6012091B7013091B801DC01CB01AC
:1030400080239123A223B3238093B5019093B601EB
:10305000A093B701B093B8011F910F910C94231462
:103060000F931F930091B5011091B6012091B70104
:103070003091B801DC01CB0180279127A227B3272B
:103080008093B5019093B601A093B701B093B801B6
:103090001F910F910C9423141092B1011092B20160
:1030A0001092B3011092B4010C94231441E050E04B
:1030B00060E070E004C0440F551F661F771F8A95BB
:1030C000D2F74093B1015093B2016093B301709372
:1030D000B4010C94231441E050E060E070E004C0BF
:1030E000440F551F661F771F8A95D2F78091B10153
:1030F0009091B201A091B301B091B401482B592B2A
:103100006A2B7B2B4093B1015093B2016093B301C2
:103110007093B4010C94231441E050E060E070E03F
:1031200004C0440F551F661F771F8A95D2F740953C
:103130005095609570958091B1019091B201A091E8
:10314000B301B091B401482359236A237B234093F0
:10315000B1015093B2016093B3017093B4010C9428
:10316000231441E050E060E070E004C0440F551FBC
:10317000661F771F8A95D2F78091B1019091B201B5
:10318000A091B301B091B401482759276A277B2742
:103190004093B1015093B2016093B3017093B401B5
:1031A0000C9423140F931F930091B1011091B2015D
:1031B0002091B3013091B401DC01CB01802B912B24
:1031C000A22BB32B8093B1019093B201A093B301D2
:1031D000B093B4011F910F910C9423140F931F937C
:1031E0000091B1011091B2012091B3013091B4016D
:1031F000DC01CB0180239123A223B3238093B1016F
:103200009093B201A093B301B093B4011F910F91B9
:103210000C9423140F931F930091B1011091B201EC
:103220002091B3013091B401DC01CB0180279127BB
:10323000A227B3278093B1019093B201A093B30169
:10324000B093B4011F910F910C9423140895CF9261
:10325000DF92EF92FF920F931F93CF93DF938C0136
:10326000C090B101D090B201E090B301F090B401F0
:103270008091B5019091B601A091B701B091B801CC
:10328000C82AD92AEA2AFB2ACFE1D0E0D701C60111
:103290000C2E04C0B695A795979587950A94D2F7FA
:1032A00080FF07C0B8018C2F0E947C0681309105F9
:1032B00031F4219758F7B80180E00E947C06DF9135
:1032C000CF911F910F91FF90EF90DF90CF900895D5
:1032D00090910C019923F1F090910D019923D1F077
:1032E000982F9695969596959F3080F5E0910E01D2
:1032F000F0910F01E90FF11D877021E030E0A90185
:1033000002C0440F551F8A95E2F7CA019181892BAB
:103310008183089520910E0130910F01F9013296B9
:103320009FEF40E05191851789F09F3F19F45111AB
:1033300001C0942F4F5F4E30A9F79F3F39F0F9013C
:10334000E90FF11D97FDFA958283089508959091F4
:103350000C019923F9F090910D019923D9F0982F40
:103360009695969596959F3028F5E0910E01F091EF
:103370000F01E90FF11D877021E030E0A90102C0C3
:10338000440F551F8A95E2F7CA01809591818923E0
:103390008183089520910E0130910F01F901329639
:1033A000205F3F4F9081891301C010823196E21750
:1033B000F307C1F7089581E090E0E0910E01F091EC
:1033C0000F01E80FF91F1082019680319105A9F7CE
:1033D00008959091CC01892B8093CC01089580951C
:1033E0009091CC0189238093CC0108951092CC0157
:1033F00008959091CB01892B8093CB0108958095FE
:103400009091CB0189238093CB0108951092CB0139
:1034100008959091CA01892B8093CA0108958095DF
:103420009091CA0189238093CA0108951092CA011C
:1034300008958093B90108951092B901089580917B
:103440000E0190910F01FC0131969C01205F3F4FCE
:1034500080E0919191118F5FE217F307D1F7089502
:10346000E0910E01F0910F018091CC018083E091F9
:103470000E01F0910F0190818091CB01892B808307
:10348000E0910E01F0910F0190818091CA01892B8A
:1034900080838091B901882361F0E0910E01F09161
:1034A0000F019081892B80830E941F1A8111109235
:1034B000B90180910E0190910F010C94D30ECF921F
:1034C000DF92EF92FF926C01EE24FF24C114D1042D
:1034D000E104F10421F0C701B60120E101C020E0C0
:1034E000C72ED82EE92EFF24C114D104E104F10423
:1034F00019F0285FC701B6016B017C0154E0F69416
:10350000E794D794C7945A95D1F7C114D104E10434
:10351000F10419F02C5FC701B6016B017C0142E098
:10352000F694E794D794C7944A95D1F7C114D1047F
:10353000E104F10419F02E5FC701B601DC01CB01F3
:10354000B695A79597958795892B8A2B8B2B09F094
:103550002F5F822FFF90EF90DF90CF9008958091A2
:10356000E501843011F120E488E190E00FB6F89491
:10357000A895809360000FBE2093600083B7817F81
:10358000846083BF83B7816083BF7894889583B755
:103590008E7F83BF0FB6F894A895809160008861F4
:1035A00080936000109260000FBE089508950C94FF
:1035B000D61ACF930E94D71A0E949B040E94D61A53
:1035C000C0E08C2F0E949105811104C0CF5FCE30E6
:1035D000C1F701C081E0CF9108950E9437140E9485
:1035E000C70E0C94BC0782E084BD93E095BD9AEFB2
:1035F00097BD80936E0008952FB7F8948091CE0107
:103600009091CF01A091D001B091D1012FBF089529
:10361000CF92DF92EF92FF920F931F932FB7F89400
:103620004091CE015091CF016091D0017091D101B4
:103630002FBF6A017B01EE24FF248C0120E030E0E3
:10364000C016D106E206F30610F4415051099A0162
:10365000281B390BC9011F910F91FF90EF90DF904C
:10366000CF9008951F920F920FB60F9211248F934F
:103670009F93AF93BF938091CE019091CF01A09182
:10368000D001B091D1010196A11DB11D8093CE0151
:103690009093CF01A093D001B093D101BF91AF918E
:1036A0009F918F910F900FBE0F901F9018950E94C1
:1036B000BF0BF8942FEF87EA91E6215080409040AD
:1036C000E1F700C0000087E090EBDC018093EE01A1
:1036D0009093EF01A093F001B093F1019CE088E199
:1036E0000FB6F894A895809360000FBE9093600089
:1036F000FFCFEF92FF920F931F93CF93DF93D82FBB
:10370000C0E08C2F0E94910500E010E0E82EF12C23
:10371000C701002E02C0959587950A94E2F780FDB7
:1037200006C00F5F1F4F0630110591F709C0602FCB
:103730007C2F80E00E9459068D13F3CF81E004C0F6
:10374000CF5FCE30F1F680E0DF91CF911F910F91E6
:10375000FF90EF900895CF93C82F8CE20E94791BC1
:10376000882321F08C2FCF910C94791B80E0CF918E
:103770000895CF930E94001D811102C00E94E61C93
:10378000C5E6C15049F00E949B048FE39CE9019774
:10379000F1F700C00000F5CF89E20E94AB1B811158
:1037A00013C18AE20E94AB1B81110E94E61C85E0D6
:1037B0000E94AB1B81110E94571B0E940B1D80931E
:1037C000CD0187E00E94AB1B8823A9F18BE10E9409
:1037D000AB1B882351F08091CD0181FB222720F97A
:1037E00091E0922790FB81F90EC08EE00E94AB1B06
:1037F000882361F08091CD0182FB222720F991E09E
:10380000922790FB82F98093CD0115C080E10E9440
:10381000AB1B9091CD01882341F093FB222720F927
:1038200081E0822780FB93F904C0892F809580FB7B
:1038300090F99093CD018091CD010E940F1D0E94BF
:103840001D1D8093DF0180EE0E94AB1B882341F099
:103850008091DF01982F909590FB80F98093DF0194
:1038600089E30E94AB1B882359F08091DF0181FB23
:10387000222720F991E0922790FB81F98093DF01C4
:1038800082EE0E94AB1B882359F08091DF0182FBFE
:10389000222720F991E0922790FB82F98093DF01A3
:1038A00086EE0E94AB1B882359F08091DF0183FBD9
:1038B000222720F991E0922790FB83F98093DF0182
:1038C00083EE0E94AB1B882359F08091DF0184FBBB
:1038D000222720F991E0922790FB84F98093DF0161
:1038E00085E30E94AB1B882359F08091DF0185FBA3
:1038F000222720F991E0922790FB85F98093DF0140
:1039000081E30E94AB1B882359F08091DF0186FB85
:10391000222720F991E0922790FB86F98093DF011E
:1039200081E10E94AB1B882359F08091DF0187FB66
:10393000222720F991E0922790FB87F98093DF01FD
:103940008091DF010E94211D8091DF0187FB882784
:1039500080F980930D0187E20E94AB1BC82F8EE196
:103960000E94AB1B8111C2608FE10E94AB1B8111D1
:10397000C46080E20E94AB1B8111C86081E20E949A
:10398000AB1B8111C06182E20E94AB1B8111C0623E
:1039900083E20E94AB1B8111C06484E20E94AB1BD6
:1039A000882311F0C06802C0CC2329F08C2F0E941C
:1039B000181D6C2F03C00E94141D682F70E080E05A
:1039C00090E0CF910C94EE17CF9108956DEE7EEFBD
:1039D00080E090E00E945A2360E082E090E00E9444
:1039E0004C2360E083E090E00E944C2360E084E0A0
:1039F00090E00E944C2360E085E090E00C944C2322
:103A000080E090E00E94462321E08D3E9E4F09F029
:103A100020E0822F089582E090E00C943E23682FEE
:103A200082E090E00C944C2383E090E00C943E23E1
:103A3000682F83E090E00C944C2384E090E00C9499
:103A40003E23682F84E090E00C944C238091D401B5
:103A500080FF0BC06091130185E0689FB0011124C5
:103A600075956795759567952BC081FF09C0609125
:103A7000130185E0689FB00111247595679520C0FA
:103A800082FF07C06091130185E0689FB001112497
:103A900017C09091D5019923D1F06091120196172A
:103AA00088F72091130185E0289F90011124929FAF
:103AB000A001939F500D112470E0CA010E941023B1
:103AC0006038710540F46115710519F406C065E0B0
:103AD00070E0862F08958FE7089581E00895809122
:103AE000D40180FF08C06091110170E07595679561
:103AF0007595679521C081FF06C06091110170E046
:103B00007595679519C082FF04C06091110170E03E
:103B100010C09091D501992399F0609110019617EA
:103B2000A0F780911101899FC001112470E00E94CB
:103B300010236038710540F46115710519F406C051
:103B400061E070E0862F08958FE7089581E0089581
:103B5000803F21F40E94261D819504C0813F29F4F5
:103B60000E94261D8093D8010895823F21F40E946F
:103B7000261D819504C0833F29F40E94261D809351
:103B8000D7010895893F19F40E946F1D05C08A3F2F
:103B900031F40E946F1D81958093D90108958B3F68
:103BA00021F40E946F1D819504C08C3F29F40E946E
:103BB0006F1D8093DA010895843F21F48091D6012E
:103BC000816017C0853F21F48091D601826011C0C9
:103BD000863F21F48091D60184600BC0873F21F499
:103BE0008091D601886005C0883F31F48091D6016C
:103BF00080618093D60108958D3F21F48091D40196
:103C000081600BC08E3F21F48091D401826005C099
:103C10008F3F29F48091D40184608093D40108956A
:103C2000803F39F48091D80187FF6CC01092D80191
:103C300069C0813F29F48091D8011816BCF362C095
:103C40009091D701823F29F497FF5CC01092D70171
:103C500059C0833F19F41916CCF354C0893F41F47D
:103C60008091D90118160CF04DC01092D9014AC0AC
:103C70008A3F29F48091D90187FF44C0F6CF8B3F5A
:103C800039F48091DA0187FF3DC01092DA013AC021
:103C90008C3F29F48091DA011816BCF333C0843FBD
:103CA00021F48091D6018E7F17C0853F21F4809149
:103CB000D6018D7F11C0863F21F48091D6018B7F84
:103CC0000BC0873F21F48091D601877F05C0883FD4
:103CD00031F48091D6018F7E8093D60113C08D3F41
:103CE00021F48091D4018E7F0BC08E3F21F480910E
:103CF000D4018D7F05C08F3F29F48091D4018B7F43
:103D00008093D4018091D70181110EC08091D80198
:103D100081110AC08091D901811106C08091DA0118
:103D2000811102C01092D501089586ED91E00E94A4
:103D3000DE0E0E94FC1A9093D3018093D201089565
:103D40001F93CF93DF938091D2019091D3010E9472
:103D5000081BAC019091D501992321F02091140109
:103D600030E006C0209115018AE0289F90011124BF
:103D70004217530708F485C08091D701C091D8013C
:103D8000D091D9011091DA01811107C0C11175C01C
:103D9000D11173C0111171C074C09F3F19F09F5FA2
:103DA0009093D501181624F40E94261D8093D70104
:103DB0008091D70187FF05C00E94261D81958093C1
:103DC000D7011C1624F40E94261D8093D8018091EF
:103DD000D80187FF05C00E94261D81958093D801D8
:103DE0006091D701662331F1C091D801CC2311F144
:103DF000062E000C770B880B990B0E94172223E3E9
:103E000033E343E35FE30E947B220E94DF21609360
:103E1000D7016C2FCC0F770B880B990B0E941722C0
:103E200023E333E343E35FE30E947B220E94DF212D
:103E30006093D8011D1624F40E946F1D8093D90150
:103E40008091D90187FF05C00E946F1D81958093E5
:103E5000D901111624F40E946F1D8093DA0180911C
:103E6000DA0187FF05C00E946F1D81958093DA01FA
:103E7000DF91CF911F910C94951E9F3F09F08FCF3A
:103E8000A0CFDF91CF911F910895E6EDF1E085E09D
:103E9000DF011D928A95E9F71092D5011092D401A5
:103EA0000895833081F128F4813059F08230D1F0C7
:103EB0000895853009F449C0B8F1863009F456C038
:103EC000089580911501262F30E0280F311D2F3FD6
:103ED000310524F4680F6093150108958FEF8093E6
:103EE0001501089580911401262F30E0280F311D0F
:103EF0002F3F310524F4680F6093140108958FEF6C
:103F000080931401089580911301262F30E0280F2B
:103F1000311D2F3F310524F4680F6093130108957C
:103F20008FEF80931301089580911201262F30E0C6
:103F3000280F311D2F3F310524F4680F60931201C3
:103F400008958FEF80931201089580911101262F1B
:103F500030E0280F311D2F3F310524F4680F6093A6
:103F6000110108958FEF8093110108958091100140
:103F7000262F30E0280F311D2F3F310524F4680F24
:103F80006093100108958FEF80931001089583309E
:103F900011F128F4813049F0823091F00895853094
:103FA00081F120F18630C1F10895809115016817E3
:103FB00020F4861B80931501089510921501089531
:103FC00080911401681720F4861B809314010895D2
:103FD00010921401089580911301681720F4861B34
:103FE0008093130108951092130108958091120196
:103FF000681720F4861B8093120108951092120115
:10400000089580911101681720F4861B8093110197
:10401000089510921101089580911001681720F4FD
:10402000861B8093100108951092100108950F933C
:104030001F938D3109F46BC008F03FC08E3009F436
:104040007DC0C0F4873009F46EC068F4863009F092
:10405000AFC08091CD01817F8E7F8093CD0181E0C3
:104060008093DC01A6C0883009F458C08B3009F475
:104070009BC09EC0863109F497C078F4803109F462
:1040800070C0813109F094C00E94371490910D01E5
:1040900081E0892780930D0187C0893109F484C0AC
:1040A0008B3109F085C08091CD0181FB222720F959
:1040B00091E0922790FB81F94AC0853309F45BC0F7
:1040C00048F4873209F457C008F45AC0893209F419
:1040D00052C06EC0833438F48A3308F067C0883326
:1040E00009F462C065C0833409F445C0883409F01E
:1040F0005FC00E9437140FEF13ED20E30150104012
:104100002040E1F700C000000E94571B4DC00E94F4
:1041100099210E94C70E0E94BC0746C00E940B1D39
:104120000E941D1D41C09091CD01892F817090FF8B
:1041300012C0917F9E7F9093CD013BC08091CD01B5
:1041400082FB222720F991E0922790FB82F980934D
:10415000CD01992349F18091CD0181608093CD01FA
:1041600023C08091CD0183FB222720F991E0922783
:1041700090FB83F9ECCF61E070E080E090E010C04C
:104180008D5141E050E060E070E08A019B0104C085
:10419000000F111F221F331F8A95D2F7C901B801E2
:1041A0000E94EE170E94371481E003C08953E9CFC3
:1041B00080E01F910F91089580E008950C94DC2019
:1041C000CF93C82F8091DC01813079F018F08230D4
:1041D000E9F187C0E0910E01F0910F0180818131FA
:1041E00069F0823209F07FC009C0E0910E01F091C0
:1041F0000F018081813111F0823261F48C2F0E9495
:10420000DE20811104C08C2F0E9417201DC081E088
:1042100090E01AC08C2F0E94DC20811114C0C431A0
:1042200079F048F4CB3079F0C03109F060C082E019
:104230008093DC0108C0C93219F0C83321F057C09F
:104240001092DC0154C081E0817053C0C93289F101
:1042500018F5C43171F1A8F4C73009F046C08AE0FE
:104260008093150194E19093140193E090931301CE
:104270008093120188E08093110188E280931001FD
:1042800034C0CE51C63088F5EC2FF0E0E65DFE4F2D
:1042900080818093DB0129C0CE34E9F020F4CB3457
:1042A00021F56AE013C0C13579F0C235F1F461E05F
:1042B0000DC08091DB01882319F01092DB0115C03D
:1042C00081E08093DC0115C061E006C08091DB01D4
:1042D0000E94511F0AC06AE08091DB010E94C71F43
:1042E00004C01092DC0180E004C081E002C080E0E4
:1042F000ABCFCF910895E1E8F0E0808188608083C2
:104300008081816080838FB7F89493E090938900D7
:1043100090ED909388008FBF0895EFE6F0E08081E4
:10432000826080830895EFE6F0E080818D7F808356
:104330000895EFE6F0E0908182E089278083089578
:104340001F920F920FB60F9211242F933F934F930A
:104350005F936F937F938F939F93AF93BF93EF93ED
:10436000FF938091DD019091DE0101969093DE0133
:104370008093DD01811103C082E00E94BC07E091BF
:10438000DE01E695E695F0E0EF5AFA4FE491809170
:10439000DD018E1303C080E00E94BC07FF91EF9106
:1043A000BF91AF919F918F917F916F915F914F914D
:1043B0003F912F910F900FBE0F901F9018950E9464
:1043C000E6216894B1110C94752208950E945A2236
:1043D00088F09F5798F0B92F9927B751B0F0E1F0C6
:1043E000660F771F881F991F1AF0BA95C9F714C076
:1043F000B13091F00E947422B1E008950C947422BF
:10440000672F782F8827B85F39F0B93FCCF38695AE
:1044100077956795B395D9F73EF49095809570950B
:1044200061957F4F8F4F9F4F0895E89409C097FB88
:104430003EF490958095709561957F4F8F4F9F4F7B
:104440009923A9F0F92F96E9BB279395F6958795BF
:1044500077956795B795F111F8CFFAF4BB0F11F482
:1044600060FF1BC06F5F7F4F8F4F9F4F16C0882329
:1044700011F096E911C0772321F09EE8872F762F5F
:1044800005C0662371F096E8862F70E060E02AF0A0
:104490009A95660F771F881FDAF7880F969587958C
:1044A00097F9089557FD9058440F551F59F05F3FF5
:1044B00071F04795880F97FB991F61F09F3F79F046
:1044C00087950895121613061406551FF2CF4695C8
:1044D000F1DF08C0161617061806991FF1CF86954A
:1044E0007105610508940895E894BB27662777272E
:1044F000CB0197F908950E948E220C94FF220E940E
:10450000F12238F00E94F82220F0952311F00C944B
:10451000E8220C94EE2211240C9475220E9452225F
:1045200070F3959FC1F3950F50E0551F629FF00106
:10453000729FBB27F00DB11D639FAA27F00DB11D1F
:10454000AA1F649F6627B00DA11D661F829F2227A8
:10455000B00DA11D621F739FB00DA11D621F839F2F
:10456000A00D611D221F749F3327A00D611D231F05
:10457000849F600D211D822F762F6A2F11249F5753
:1045800050409AF0F1F088234AF0EE0FFF1FBB1F56
:10459000661F771F881F91505040A9F79E3F510515
:1045A00080F00C94E8220C9475225F3FE4F3983E6F
:1045B000D4F3869577956795B795F795E7959F5FBF
:1045C000C1F7FE2B880F911D9695879597F9089551
:1045D00097F99F6780E870E060E008959FEF80ECB6
:1045E000089500240A941616170618060906089559
:1045F00000240A9412161306140605060895092EBF
:104600000394000C11F4882352F0BB0F40F4BF2B2D
:1046100011F460FF04C06F5F7F4F8F4F9F4F08956D
:1046200097FB072E16F4009407D077FD09D00E945F
:104630002A2307FC05D03EF4909581959F4F08955D
:10464000709561957F4F0895EE0FFF1F0590F491CF
:10465000E02D0994AA1BBB1B51E107C0AA1FBB1F79
:10466000A617B70710F0A61BB70B881F991F5A95FE
:10467000A9F780959095BC01CD010895F999FECFD9
:1046800092BD81BDF89A992780B50895A8E1B0E060
:1046900042E050E00C946123262FF999FECF1FBA17
:1046A00092BD81BD20BD0FB6F894FA9AF99A0FBE5B
:1046B000019608950E944C23272F0C944D23DC0172
:1046C000CB01FC01F999FECF06C0F2BDE1BDF89A1D
:1046D000319600B40D9241505040B8F70895F894C7
:0246E000FFCF0A
:1046E2002002BE074E082908F507C1070101BA01D9
:1046F20028080A03140A3F4D36391205C5048F04EF
:104702005604E90302041B043404010203040506EF
:04471200070809008B
:00000001FF
